:1000000013C037C036C035C034C033C032C031C071
:1000100030C02FC02EC02DC08DC02BC02AC029C01B
:1000200028C027C026C02A0111241FBECFE5D2E078
:10003000DEBFCDBF10E0A0E6B0E0E2E6F3E002C034
:1000400005900D92A236B107D9F720E0A2E6B0E004
:1000500001C01D92A037B207E1F710E0C8E2D0E07E
:1000600003C02297FE0177D1C632D107D1F7A2D0C3
:1000700076C1C6CFA4E0B0E0EFE3F0E03CC120E100
:1000800030E00090670002C0220F331F0A94E2F7AD
:10009000BFB6F894C0906200D0906300E090640016
:1000A000F0906500A90156954795640F751F811D55
:1000B000911D40E050E0F4D02C0D3D1D4E1D5F1D04
:1000C000BFBE29833A834B835C831DD0BFB6F894AF
:1000D0008091620090916300A0916400B0916500EE
:1000E00029813A814B815C8179018A01E81AF90AF8
:1000F0000A0B1B0B1E141F04100611060CF3BFBEC7
:100100002496E9E014C185B7877E85BF85B78062F4
:1001100085BF889585B78F7D85BF089520ED37E031
:10012000615071098109910920F0F9013197F1F7C6
:10013000F7CF08951F920F920FB60F9211242F93AD
:100140003F934F935F936F937F938F939F93AF935F
:10015000BF93EF93FF938091620090916300A09111
:100160006400B09165000196A11DB11D80936200ED
:1001700090936300A0936400B0936500E0916A00DF
:10018000F0916B00309729F08091680090916900A0
:100190000995FF91EF91BF91AF919F918F917F91C1
:1001A0006F915F914F913F912F910F900FBE0F90E4
:1001B0001F90189586B1866086B980E889B97894D1
:1001C0009FB7F894A89584B7877F84BF88E181BDE5
:1001D00080E481BD9FBF10926B0010926A00109264
:1001E0006900109268001092670081E080936600B9
:1001F0008AE390E090936100809360009FB7F89449
:10020000E0916C00F0916D00828120916E00822B54
:1002100082839FBFE0916000F091610060E170E037
:1002200080E090E009959FB7F894E0916C00F09120
:100230006D00228180916E008095822382839FBF12
:10024000E0916000F091610060E072E080E090E099
:100250000995D4CFCF93DF9389E390E090936D001D
:1002600080936C0080E280936E0085E080936F0045
:100270009FB7F894ECE6F0E0C081D1818981AEE6C9
:10028000B0E02C91822B89830190F081E02D2281B6
:100290008C918095822382839FBFDF91CF910895B7
:1002A000A1E21A2EAA1BBB1BFD010DC0AA1FBB1F7A
:1002B000EE1FFF1FA217B307E407F50720F0A21BEC
:1002C000B30BE40BF50B661F771F881F991F1A9459
:1002D00069F760957095809590959B01AC01BD0183
:1002E000CF0108952F923F924F925F926F927F922B
:1002F0008F929F92AF92BF92CF92DF92EF92FF9236
:100300000F931F93CF93DF93CDB7DEB7CA1BDB0BE1
:100310000FB6F894DEBF0FBECDBF09942A88398886
:1003200048885F846E847D848C849B84AA84B9848D
:10033000C884DF80EE80FD800C811B81AA81B98199
:10034000CE0FD11D0FB6F894DEBF0FBECDBFED01AD
:100350000895EE0FFF1F0590F491E02D0994F89495
:02036000FFCFCD
:020362008E000B
:00000001FF
